:020000040000FA
:1000000007309F0083169F01831212288207543401
:1000100045344D345034453420343D340034D634E6
:100020004334003432192728831685100511003017
:1000300086008312851005113830952001309520F7
:10004000033095200F309520803095203528831679
:100050008510051100308600831285100511383097
:1000600095200C309520C0309520AB203820A92851
:100070008316851005110030860083128510051146
:100080003830952001309520033095200F30952091
:1000900080309520073079208316851005110030B7
:1000A0008600831285100511383095200C3095207C
:1000B000C030952032185E28FA309A202008860039
:1000C0009A20210886009A20B218672070282E30C6
:1000D0009A2023089A2020309A200F308720080089
:1000E00020309A2020309A2020309A200F3087200C
:1000F0000800B4000630B402B40334080620B1008E
:10010000B108031986289A20B40A7D280800B40093
:100110000630B402B40334080620B100B108031954
:1001200094289A20B40A8B280800860085109F2006
:10013000B4210800860085149F20B421080005150D
:100140000000051108002F18A928360886009A20FB
:100150000800BE211228BF20D420D6202721D62077
:100160001F21BF20D420D620F220D620F428B000B2
:10017000F428AF00BF2029218C219B210800C22038
:10018000CF200800831685158312831685118312EC
:100190008511AE21831685158312A52108008519C6
:1001A000CF28851DD1280800CC300800AD000830CC
:1001B000AE0083168515831283168511831285116F
:1001C000AD0C031CE728831685158312EB288316D4
:1001D000851183128511A821831685158312AE0B14
:1001E000DC280800BE3008000830A500A6018316F0
:1001F00085158312831685118312851100008316DD
:1002000085158312A021031085190314A60CA821BB
:10021000831685158312A50BFA282608321914298E
:10022000A8003215B215B728B2191D2928020319E2
:10023000A9282608A800B215B728B211B928831634
:1002400085158312851D2229BE2100000800443037
:1002500008002F2142214C21732187210800B3017E
:100260000330AE000314AF0CB00CB30CAE0B32294C
:100270000310B00CB30C0430AE000310B30CAE0B83
:100280003D29080032100311FF302F0503194A29B8
:10029000321408003210080003110030330403192F
:1002A0006F290C30330503196329B3195A29331DFB
:1002B0005F295D29331961295F2966217129692127
:1002C00071296C2171293130A30008003330A3005B
:1002D00008003530A30008003830A3000800B21031
:1002E0000800B21408003008B501B601B7000A30A2
:1002F0003702031C8429B700B60A0A303602031CF1
:100300007729B601B50A7729360E3707080030304D
:10031000B504B604B704080032188F29FA3036083D
:10032000A0003708A100B2189629982923080800D0
:100330003030A30008002E30A20008000530B0299C
:100340000230B02903300000B02905300000B02988
:100350000F30B0291330B0291630B029A630B0299B
:10036000AA00AA0BB12908004030B629AC00FF3022
:10037000AA00AA0BB929AC0BB72908000630C0297E
:10038000AC00D930AB00FF30AA00AA0BC529AB0BDB
:08039000C329AC0BC1290800D0
:02400E00293F48
:00000001FF
